:100000000EC01DC03FC01BC01AC019C018C017C009
:1000100016C015C014C013C012C011C010C01124E6
:100020001FBECFE5D2E0DEBFCDBF20E0A0E6B0E04E
:1000300001C01D92A236B207E1F702D04DC0E0CF59
:10004000B89A8BB780628BBFA89A7894E0E6F0E00C
:10005000809160009091610001969093610080937F
:10006000600098B3892788BB98B38081892B88BBAF
:1000700098B38081892388BB88B310926100109265
:100080006000E6CF1F920F920FB60F9211248F934C
:100090009F93C49AB09B0AC08091600090916100C8
:1000A0000196909361008093600009C08091600088
:1000B000909161000197909361008093600083ECC0
:1000C00099E00197F1F700C000009F918F910F9088
:0C00D0000FBE0F901F901895F894FFCF02
:00000001FF
